:020000001229C3
:08000800822870308F001108FE
:100010009000900B09288F0B072869228E0B05286A
:10002000080010308E0010309000900B15286922C7
:100030008E0B132808000514013092000520920150
:10004000051085100E308E000520080010308E003F
:100050001C202D2810308E001B20061A1D14EA20AB
:10006000A20803190D10692208000A30B70703100F
:10007000B70D370D422830308E001C204428473001
:10008000422830308E001B20861A1D14EA20A20858
:1000900003198D10692208000310B70D370D55287C
:1000A000403055281530552820308E000510851019
:1000B0009201052008000514013092001030A200C2
:1000C0000D1010308F008D1011208D1C74280D1C08
:1000D0006D28A108031D5E287628A10803195E2853
:1000E000A20B6128A10161288F0B642892010510E1
:1000F000851010308E0005209D01EA208D106922A8
:10010000A20108008B138C00030893000B116922D5
:10011000061F2314861FA3140B189A28920803198C
:100120009C2892030319962885109C28023092007F
:1001300085149C2820308B00930E130E83008C0EA8
:100140000C0E8B17090008309C00990C031CAA2880
:1001500016089707970C980C9C0BA5280800000020
:1001600010309C00980103109A0D990D980D1608F7
:100170001802031CBE28160898020314970D9C0B46
:10018000B328080005128316FF309C000000000011
:1001900000009C0BC6280516831208009601960FD6
:1001A000D2280800051ECF2808008B13C220051591
:1001B000831605118312CE208316051505128312AE
:1001C00005128B170C309900A32017089E00180801
:1001D0009F0008008B13C22085158316851183129A
:1001E000CE20831685150512831205128B171E0863
:1001F00099001F089A00B0201708910008000830E5
:100200008B00FC3086058316061086108605831247
:100210008B17630000008B13831606148614831259
:100220008B17080085018D01A3018E019201A201A7
:10023000BB013B148316023081000C308500F33083
:1002400086008312A0308B00D520EA208615692213
:100250008D08031D3A296E22A308031D3A29D520D3
:1002600069228D08031D3A296E22A308031D3A292D
:10027000FF20EA2003300605B6002318C429A3187E
:10028000C8290319AB29B60303195229B603031968
:100290007E290D1C4D298D102A208D1C26290D101C
:1002A00041202629A001A10169220D185E298D1C7B
:1002B0002629A1010230A000412054298D1865296A
:1002C000A1010130A0002A205429A1080319702996
:1002D00020186D2941200D1054292A208D105429F1
:1002E0000130A100201879292A200130A0008D10AA
:1002F000542941200230A0000D105429A001A10171
:1003000069220D188A298D1C2629A1010230A0001E
:100310005B2080298D189229A1010130A0002A209C
:100320008D108029A10803199D2920189A295B2086
:100330000D1080292A208D1080290130A10020185D
:10034000A6292A200130A0008D1080295B200230D0
:10035000A0000D1080292A202A202A204120542084
:1003600026291030B300B529B301AA0172232B0846
:1003700008000F303A181F30A600080040309100E6
:100380005020EA20BA010800BE21061BB22ACC295F
:10039000BE213A14861BB22A3B2026202620262086
:1003A0003B20A30154208D01B921AA011030B300D4
:1003B0003A1CB3010230A7008D08031DE929A308E8
:1003C000031DE429FF20DC29AC0184233B20A30189
:1003D0002629FB30AC0084230130AA00AC01EA20BE
:1003E000061E0D140D1CFA298D10262089220038B6
:1003F000031D432A861E8D148D1C0F2A0D100230FA
:100400003602031D0A2A4C2273220038031D432A98
:1004100078220C2A3B2084220038031D432A6922BB
:100420000D18F0298D18FA29A308031D422A05305A
:10043000B800B70104308E0005208D08031D2D2A59
:10044000A308031D422AB70AB71D1A2A8E220038B4
:10045000031D432AB80B192A382AB7080319382A6A
:1004600093220038031D432A7E220038031D432AAD
:1004700069228D08031DEF29A308031D422AFF20CE
:100480006922EF29A822542026203B2026203B2049
:100490002620A3018D012629B701013092000430E6
:1004A0008E0005208D1019303702031CB70A0A3060
:1004B0008F001120861E8D148D184F2A8F0B592AFC
:1004C0009201851010308E000520EA208D106922DF
:1004D0000800061E0D14861E8D140800061F231426
:1004E000861FA3140800AC112C11AC142C14972AED
:1004F0000A30B702031CB7010F30B705F030AC0566
:100500000F303705AC04972AAC112C11AC142C1009
:10051000972AAC112C15AC102C10972AAC112C1169
:10052000AC102C10972AAC112C11AC102C14A70B6A
:10053000A62A8423AA0A031DA22AB30A3308260284
:10054000031CFF340230A700AC010034AC0E0034B1
:10055000AC112C15AC142C10A70BB02A8423080066
:10056000AC0EAC2A231CBE2AA31CB92A3B18052BAF
:10057000BB2A3B1C052BB421B921C02AB921B121CA
:10058000FB302B020319CB2A3B205420542054204B
:100590008D01A3012629B9010130AA000230A7006C
:1005A0007223A501AB0E0F302B05391CDF2AB700D3
:1005B000B918DC2A4C20DD2A3520B901F72AA5001C
:1005C000B9010310A50C031CE92A39142518B91424
:1005D000F72AA508031DEE2A5420F72AA50BF22AB4
:1005E0004120F72AA50BF62A2A20F72AC52A8D18BA
:1005F000C52AA501A70BD22AAA0A031DCE2AB30A2F
:1006000033082602031CC52ACE2A8D01A301262900
:100610008B1386158316861183128B170611000023
:100620000615000000000000000000008611000018
:10063000000000000000000006110000000008009B
:100640008B1386118316861183128B178611000077
:1006500000000000061500000000000086150000E4
:100660000000061100000000000008008B13831634
:10067000861183128B17281F3F2B8615402B86115E
:100680000615000000000000000006110800A81771
:100690008B1383168615831286150615000000003D
:1006A000000000000000861DA81306118B1708002B
:1006B0000830AF002813AE1B28173623AE0DAF0B42
:1006C0005A2B4723A81BB50A0800AB010830AF001E
:1006D0000310AB0D4723A81B2B14AF0B682B281757
:1006E00036230800B5010823A030AE005823330894
:1006F000AE0058232A08AE0058230823A130AE00CC
:100700005823652320230800B501A030AD0008233D
:100710002D08AE0058233308AE0058232A08AE0037
:0C07200058232C08AE00582320230800AA
:02400E00F13F80
:00000001FF
